S023000064656D6F70726F675F6E75636C656F5F73746D33326631303372622E73726563D9
S3150800200000500020F9270008492800084928000838
S315080020104928000849280008492800080000000047
S315080020200000000000000000000000004928000829
S3150800203049280008000000004928000891280008DF
S31508002040492800084928000849280008492800089E
S31508002050492800084928000849280008492800088E
S31508002060492800084928000849280008492800087E
S31508002070492800084928000849280008492800086E
S31508002080492800084928000849280008492800085E
S31508002090492800084928000849280008492800084E
S315080020A0492800084928000849280008492800083E
S315080020B0492800084928000849280008492800082E
S315080020C0492800084928000849280008492800081E
S315080020D0492800084928000849280008492800080E
S315080020E04928000849280008492800080000000077
S315080020F000000000000000000000000000000000D2
S3150800210000000000000000005FF808F1EE11AA5573
S3150800211010B5054C237833B9044B13B10448AFF313
S3150800212000800123237010BD140000200000000069
S31508002130E828000808B5034B1BB103490348AFF369
S31508002140008008BD0000000018000020E8280008EC
S3150800215030B587B001214FF4003000F035FA01217F
S31508002160052000F023FA18238DF817300425ADF85A
S31508002170145003238DF81630144C05A9204600F098
S3150800218063F98DF817500823ADF8143005A92046D1
S3150800219000F05AF94FF4614301930023ADF8083073
S315080021A0ADF80A30ADF80C30ADF810300C23ADF8A8
S315080021B00E30A4F544440DEB0501204600F012FA52
S315080021C00121204600F072FA07B030BD0008014030
S315080021D010B504462021064800F07AFA012801D0F5
S315080021E0002010BD024800F06FFA2070012010BDD3
S315080021F00044004008B5FFF7ABFF08BD0449CA68AC
S3150800220002F4E062034B1343CB60BFF34F8FFEE744
S3150800221000ED00E00400FA0508B5224B1B78B3B9B7
S315080022202148FFF7D5FF012800D008BD1E4B1B78B3
S31508002230013BDBB23F2BF8D800F024FB1B4B1860A0
S315080022400122184B1A700022194B1A7008BD184B38
S315080022501B78013314481844FFF7BAFF01280AD03F
S3150800226000F010FB114B1B6864339842DDD900223D
S315080022700C4B1A70D9E70E4A13780133DBB2137088
S31508002280094A12789342D0D10022064B1A70064B9F
S315080022905B78FF2BC9D1044B9B78002BC5D1FFF780
S315080022A0ADFF00BF71000020300000207400002040
S315080022B07200002008B5FFF7AFFF08BD00B583B070
S315080022C00121042000F072F92023ADF8043003231D
S315080022D08DF8063010238DF8073001A9024800F062
S315080022E0B3F803B05DF804FB0008014010B500F030
S315080022F0C9FA0E4B1B68C31AB3F5FA7F0CD304460A
S315080023000B4B1B784BB90122094B1A70202109483F
S3150800231000F0E9F8054B1C6010BD0022044B1A704A
S315080023202021044800F0E1F8F4E700BF7C00002013
S31508002330780000200008014082B000230193009332
S315080023402C4A136843F4803313602A4B1B6803F442
S3150800235000330093019B01330193009B1BB9019B3A
S31508002360B3F5A06FF1D1234B1B6813F4003F06D0D9
S3150800237001230093009B012B04D002B07047002371
S315080023800093F7E71C4B1A6842F010021A601A68A5
S3150800239022F003021A601A6842F002021A60A3F5D4
S315080023A080535A685A605A685A605A6842F480627A
S315080023B05A605A6822F47C125A605A6842F4E81243
S315080023C05A601A6842F080721A600A4B1B6813F04A
S315080023D0007FFAD0074B5A6822F003025A605A68FF
S315080023E042F002025A60034B5B6803F00C03082BA9
S315080023F0F9D1C2E7001002400020024008B5FFF7F5
S315080024009BFF08BD08B50E4B1A6842F001021A6018
S3150800241059680C4A0A405A601A6822F0847222F4F3
S3150800242080321A601A6822F480221A605A6822F4E6
S31508002430FE025A604FF41F029A60FFF7DFFF08BDDD
S31508002440001002400000FFF8F0B4CB7803F00F024A
S31508002450154613F0100F01D08D7815430B78E3B1AC
S315080024600668002301E042610133072B14D80122D4
S315080024709A400C8832EA0404F6D19C000F27A7403C
S3150800248026EA070605FA04F42643CC78282CEAD06F
S31508002490482CE9D10261E7E706600B88FF2B20D9B3
S315080024A04668002302E0426115E00133072B17D87E
S315080024B003F108040122A2400C8832EA0404F4D18C
S315080024C09C000F27A74026EA070605FA04F42643C8
S315080024D0CC78282CE7D0CC78482CE6D10261E4E702
S315080024E04660F0BC70470161704741617047000063
S315080024F010B4294B5B6803F00C03042B2BD0082B74
S315080025002CD013B1254B036001E0244B036022490C
S315080025104B68C3F30313224CE35CDAB20368D34077
S3150800252043604A68C2F30222A25CD2B223FA02F2DC
S3150800253082604A68C2F3C222A25CD2B2D340C360A8
S315080025404A68C2F3813217498A5CD2B2B3FBF2F306
S31508002550036110BC7047114B0360D8E70E4A5368F5
S315080025605268C3F38343023312F4803F09D00A4A00
S31508002570526812F4003F09D00B4A02FB03F30360CA
S31508002580C5E7094A02FB03F30360C0E7034A02FBF7
S3150800259003F30360BBE700BF0010024000127A0095
S315080025A0040000200000002000093D0029B9054A62
S315080025B0936923EA000090617047024A93691843B9
S315080025C0906170470010024029B9054AD36923EA89
S315080025D00000D0617047024AD3691843D06170473A
S315080025E00010024030B587B004460D46038A9BB2F8
S315080025F0CA8823F440531343038283899BB289888C
S3150800260028896A8901430A4323F4B05323F00C034B
S315080026101343A381A38A9BB2AA8923F44073134365
S31508002620A38201A8FFF764FF1E4B9C4224D0039B9C
S31508002630A28912F4004F21D103EB830303EB830332
S3150800264029688900B3FBF1F1174BA3FB012358094D
S315080026500501642300FB1313A28912F4004F16D157
S315080026601B013233104AA2FB0323C3F343132B4344
S315080026709BB2238107B030BD049BD9E703EB8303E4
S3150800268003EB830329684900B3FBF1F1DCE7D900C2
S315080026903231054AA2FB0131C1F3421245EA02036F
S315080026A0E6E700BF003801401F85EB5131B9838941
S315080026B09BB223F400539BB28381704783899BB2F4
S315080026C043F40053838170478088C0F3080070473D
S315080026D00388194201D10020704701207047000085
S315080026E000B583B000230193009303F1804303F5FB
S315080026F004331A6842F001021A605968364A0A40D9
S315080027005A601A6822F0847222F480321A601A68B3
S3150800271022F480221A605A6822F4FE025A604FF4A4
S315080027201F029A601A6842F480321A602B4B1B68A3
S3150800273003F400330093019B01330193009B23B9F3
S31508002740019A40F2DC539A42F0D1244B1B6813F4E9
S31508002750003F00D1FEE7224B1A6842F010021A60C9
S315080027601A6822F003021A601A6842F002021A6016
S31508002770A3F580535A685A605A6842F400525A6060
S315080027805A6842F480625A605A6822F47C125A6087
S315080027905A6842F4E8125A601A6842F080721A605F
S315080027A00E4B1B6813F0007FFAD00C4B5A6822F0C8
S315080027B003025A605A6842F002025A60074B5B6885
S315080027C003F00C03082BF9D1FFF778FD00F044F865
S315080027D003B05DF804FB00BF0000FFF800100240DC
S315080027E00020024008B5FFF77BFFFFF703FDFFF760
S315080027F07DFDFFF75FFDFAE7DFF834D0002103E03F
S315080028000C4B5B58435004310B480C4B42189A4208
S31508002810F6D30B4A02E0002342F8043B094B9A42DE
S31508002820F9D3FFF7EFFD00F03BF8FFF7DBFF704742
S31508002830005000200829000800000020140000208D
S315080028401400002084000020FEE70000014B1860F9
S31508002850704700BF8000002008B5074B074A5A603A
S31508002860F021074A82F823100020986007221A6090
S31508002870FFF7ECFF08BD00BF10E000E03F190100BC
S3150800288000ED00E0014B1868704700BF800000208B
S31508002890024A136801331360704700BF80000020A6
S315080028A070B500250C4E0D4CA41BA410A54209D1E9
S315080028B000F01AF800250A4E0A4CA41BA410A542DB
S315080028C005D170BD56F8253098470135EEE756F81C
S315080028D0253098470135F2E7002900080029000845
S315080028E00029000804290008F8B500BFF8BC08BC90
S315080028F09E467047F8B500BFF8BC08BC9E467047B0
S309080029003521000867
S309080029041121000887
S315080029080204060800000000010203040102030489
S30908002918060708098F
S705080027F9D2
